:020000040000FA
:100000008A110A1208280000000000000000000009
:10001000283084005830A0008001840AA00B0C28EE
:10002000103095002730960000308E0000308F0091
:10003000013090000B30970007309F0000308500A2
:100040008316FD3085008312003086008316D7307A
:10005000860083120C1D2A280C116400A914A9180B
:100060002915A91C2911851936282911291D3A2875
:10007000A9113B28A915A9182915A91C2911A919E5
:1000800042282911291D592800302B0203194F2815
:10009000A00020092B05A006A01B542858283130A9
:1000A0002A02031C54285828AA0F5728AB0A2911E2
:1000B0005D280030AA000030AB00291D60282916F9
:1000C000A9182915A91C2911A91229192917291DAF
:1000D0002913A91B6C282913291F6F28A916291970
:1000E0002917291D2913A91976282913291F7928C9
:1000F000A916A91A2915A91E291129192C14291D77
:100100002C10AC1C842829112C18AC142C1CAC10FD
:10011000291D8B282912A9182915A91C29112C1170
:100120002919AC15291DAC11291A9728AC11AC1D41
:100130009A282C152919AC15291DAC112C1AA128A7
:10014000AC11AC1DA4282C152C1929152C1D291116
:1001500029198616291D8612A9182915A91C2911E5
:10016000051AB3282911291DB728A913B828A917DA
:10017000A9182915A91C2911A91BBF282911291D56
:10018000D62800302E020319CC28A00020092E0505
:10019000A006A01BD128D52831302D02031CD12860
:1001A000D528AD0FD428AE0A2911DA280030AD00C9
:1001B0000030AE00291DDD28AC16A9182915A91C90
:1001C00029112C132919AC17291DAC13A919E928D9
:1001D000AC13AC1FEC282C172919AC17291DAC1334
:1001E000A91BF328AC13AC1FF6282C172C1B2915C0
:1001F0002C1F291129192C14291D2C102F1C012901
:1002000029112C182F142C1C2F10291D0829AC1271
:10021000A9182915A91C2911AF1029192F15291D55
:100220002F11AC1A14292F112F1D1729AF142919BA
:100230002F15291D2F112C1A1E292F112F1D212991
:10024000AF14AF182915AF1C291129198615291DBE
:100250008611A9182915A91C2911291A3029291133
:10026000AC1A33292911291D36292C16A91829154C
:10027000A91C2911AF1129192F16291D2F12A919EF
:1002800042292F122F1E4529AF1529192F16291D76
:100290002F12A91B4C292F122F1E4F29AF15AF1952
:1002A0002915AF1D291129192C14291D2C10AF1E39
:1002B0005A2929112C18AF162C1CAF12291D61299F
:1002C0002C12A9182915A91C29112F1F68292911D9
:1002D000291D7F290030310203197529A00020094A
:1002E0003105A006A01B7A297E2927303002031C85
:1002F0007A297E29B00F7D29B10A2911832900307E
:10030000B0000030B100AF1B89292730B2000030A7
:10031000B300AF172919A129003033020319972917
:10032000A00020093305A006A01B9C29A029273086
:100330003202031C9C29A029B20F9F29B30A291558
:10034000A5290030B2000030B30029192F17291D4C
:100350002F13A9182915A91C29112C1AB029291104
:100360002F1BB329291129198514291D85108A01EC
:020370002A2839
:02400E00623F0F
:00000001FF
